:020000040000FA
:100000000528BF28BF28BF286D28030183018B0165
:1000100085018601FF30860091017F309400143005
:1000200095000130CD009601831610308500013017
:100030008600D330810083120B168B17051E2B28E8
:10004000CD0B2828DF308600FF3086000B30CD0036
:10005000FF30C5201E280130CD0003301102031DE2
:10006000392886010C30C520FF3086001508C520D0
:100070001E2802301102031D3F2886016628013028
:100080001102031D46281408860066280430110258
:10009000031D642800220038031D54289601FF30F8
:1000A000C520FF30C5201E288601C520960A0022E3
:1000B0000038031D5D289601BF209000FF308600A8
:1000C0001008C520960A1E28FF3086000B1D6A28DE
:1000D00085146300000000001E28C000030E830189
:1000E000C1004E08CF0085108B1CBF281430C520DE
:1000F000061CB728051AB72882309300061C9228E0
:1001000000000000930F7E2803011104031D9028B6
:10011000910A7F30940096018B1281010B11B72850
:100120009101B728030111040319B7280B19A0285E
:10013000910A053011020318910181010B11B728B2
:1001400001301102031DAB280310940C9419AA2846
:100150007F309400B72803301102031DB7282830E0
:1001600015020318B5289503B7280A3095028B109D
:100170004F08CE00410E8300C00E400E0900051549
:100180008B01000000000000C128CE00CE0BC92862
:0C01900008000000000000000000C6286D
:1004000002308A0016081F3982071E3478341E34E1
:1004100078341E34F034783478347834783478345E
:10042000F0341E3478341E3478341E34FF340034F3
:1004300000000000000000000000000000000000BC
:1004400000000000000000000000000000000000AC
:0604500000000000003472
:02400E00F33F7E
:00000001FF
